 jimage

 Timestamp is 5d1c9e51 (reproducible build file hash)

 Preferred load address is 10000000

 Start         Length     Name                   Class
 0001:00000000 00000020H .text$di                CODE
 0001:00000020 0000249dH .text$mn                CODE
 0002:00000000 000000f8H .idata$5                DATA
 0002:000000f8 00000008H .00cfg                  DATA
 0002:00000100 00000004H .CRT$XCA                DATA
 0002:00000104 00000008H .CRT$XCU                DATA
 0002:0000010c 00000004H .CRT$XCZ                DATA
 0002:00000110 00000004H .CRT$XIA                DATA
 0002:00000114 00000004H .CRT$XIZ                DATA
 0002:00000118 00000004H .CRT$XPA                DATA
 0002:0000011c 00000004H .CRT$XPZ                DATA
 0002:00000120 00000004H .CRT$XTA                DATA
 0002:00000124 00000004H .CRT$XTZ                DATA
 0002:00000128 00000000H .gfids$y                DATA
 0002:00000128 000002d8H .rdata                  DATA
 0002:00000400 00000000H .rdata$CastGuardVftablesA DATA
 0002:00000400 00000000H .rdata$CastGuardVftablesC DATA
 0002:00000400 000002c4H .rdata$r                DATA
 0002:000006c4 00000004H .rdata$sxdata           DATA
 0002:000006c8 00000064H .rdata$voltmd           DATA
 0002:0000072c 000002fcH .rdata$zzzdbg           DATA
 0002:00000a28 00000004H .rtc$IAA                DATA
 0002:00000a2c 00000004H .rtc$IZZ                DATA
 0002:00000a30 00000004H .rtc$TAA                DATA
 0002:00000a34 00000004H .rtc$TZZ                DATA
 0002:00000a38 00000118H .xdata$x                DATA
 0002:00000b50 00000124H .edata                  DATA
 0002:00000c74 0000008cH .idata$2                DATA
 0002:00000d00 00000014H .idata$3                DATA
 0002:00000d14 000000f8H .idata$4                DATA
 0002:00000e0c 000004d0H .idata$6                DATA
 0003:00000000 00000028H .data                   DATA
 0003:00000028 00000060H .data$r                 DATA
 0003:00000088 000000d8H .data$rs                DATA
 0003:00000160 000003a4H .bss                    DATA
 0004:00000000 00000060H .rsrc$01                DATA
 0004:00000060 00000328H .rsrc$02                DATA

  Address         Publics by Value              Rva+Base       Lib:Object

 0000:00000000       ___AbsoluteZero            00000000     <absolute>
 0000:00000000       ___arm64x_extra_rfe_table  00000000     <absolute>
 0000:00000000       ___arm64x_extra_rfe_table_size 00000000     <absolute>
 0000:00000000       ___arm64x_native_entrypoint 00000000     <absolute>
 0000:00000000       ___arm64x_redirection_metadata 00000000     <absolute>
 0000:00000000       ___arm64x_redirection_metadata_count 00000000     <absolute>
 0000:00000000       ___dynamic_value_reloc_table 00000000     <absolute>
 0000:00000000       ___enclave_config          00000000     <absolute>
 0000:00000000       ___guard_check_icall_a64n_fptr 00000000     <absolute>
 0000:00000000       ___guard_eh_cont_count     00000000     <absolute>
 0000:00000000       ___guard_eh_cont_table     00000000     <absolute>
 0000:00000000       ___guard_fids_count        00000000     <absolute>
 0000:00000000       ___guard_fids_table        00000000     <absolute>
 0000:00000000       ___guard_iat_count         00000000     <absolute>
 0000:00000000       ___guard_iat_table         00000000     <absolute>
 0000:00000000       ___guard_longjmp_count     00000000     <absolute>
 0000:00000000       ___guard_longjmp_table     00000000     <absolute>
 0000:00000000       ___hybrid_auxiliary_delayload_iat 00000000     <absolute>
 0000:00000000       ___hybrid_auxiliary_delayload_iat_copy 00000000     <absolute>
 0000:00000000       ___hybrid_auxiliary_iat    00000000     <absolute>
 0000:00000000       ___hybrid_auxiliary_iat_copy 00000000     <absolute>
 0000:00000000       ___hybrid_code_map         00000000     <absolute>
 0000:00000000       ___hybrid_code_map_count   00000000     <absolute>
 0000:00000000       ___hybrid_image_info_bitfield 00000000     <absolute>
 0000:00000000       ___x64_code_ranges_to_entry_points 00000000     <absolute>
 0000:00000000       ___x64_code_ranges_to_entry_points_count 00000000     <absolute>
 0000:00000001       ___safe_se_handler_count   00000001     <absolute>
 0000:00000100       ___guard_flags             00000100     <absolute>
 0000:00000000       ___ImageBase               10000000     <linker-defined>
 0001:00000020       ?map_size@ImageFileReader@@QBE_KXZ 10001020 f i NativeImageBuffer.obj
 0001:00000036       _Java_jdk_internal_jimage_NativeImageBuffer_getNativeMap@12 10001036 f   NativeImageBuffer.obj
 0001:00000088       ?get@NativeEndian@@UAEFF@Z 10001088 f   endian.obj
 0001:00000088       ?get@NativeEndian@@UAEGG@Z 10001088 f   endian.obj
 0001:00000090       ?get@NativeEndian@@UAEHH@Z 10001090 f   endian.obj
 0001:00000090       ?get@NativeEndian@@UAEII@Z 10001090 f   endian.obj
 0001:00000097       ?get@NativeEndian@@UAE_J_J@Z 10001097 f   endian.obj
 0001:00000097       ?get@NativeEndian@@UAE_K_K@Z 10001097 f   endian.obj
 0001:000000a2       ?set@NativeEndian@@UAEXAAFF@Z 100010a2 f   endian.obj
 0001:000000a2       ?set@NativeEndian@@UAEXAAGG@Z 100010a2 f   endian.obj
 0001:000000b1       ?set@NativeEndian@@UAEXAAHH@Z 100010b1 f   endian.obj
 0001:000000b1       ?set@NativeEndian@@UAEXAAII@Z 100010b1 f   endian.obj
 0001:000000be       ?set@NativeEndian@@UAEXAA_J_J@Z 100010be f   endian.obj
 0001:000000be       ?set@NativeEndian@@UAEXAA_K_K@Z 100010be f   endian.obj
 0001:000000d2       ?get@SwappingEndian@@UAEFF@Z 100010d2 f   endian.obj
 0001:000000d2       ?get@SwappingEndian@@UAEGG@Z 100010d2 f   endian.obj
 0001:000000de       ?get@SwappingEndian@@UAEHH@Z 100010de f   endian.obj
 0001:000000de       ?get@SwappingEndian@@UAEII@Z 100010de f   endian.obj
 0001:000000e7       ?get@SwappingEndian@@UAE_J_J@Z 100010e7 f   endian.obj
 0001:000000e7       ?get@SwappingEndian@@UAE_K_K@Z 100010e7 f   endian.obj
 0001:000000fa       ?set@SwappingEndian@@UAEXAAFF@Z 100010fa f   endian.obj
 0001:000000fa       ?set@SwappingEndian@@UAEXAAGG@Z 100010fa f   endian.obj
 0001:0000010d       ?set@SwappingEndian@@UAEXAAHH@Z 1000110d f   endian.obj
 0001:0000010d       ?set@SwappingEndian@@UAEXAAII@Z 1000110d f   endian.obj
 0001:0000011c       ?set@SwappingEndian@@UAEXAA_J_J@Z 1000111c f   endian.obj
 0001:0000011c       ?set@SwappingEndian@@UAEXAA_K_K@Z 1000111c f   endian.obj
 0001:00000138       ?get_handler@Endian@@SAPAV1@_N@Z 10001138 f   endian.obj
 0001:0000014b       ?get_java@Endian@@SAGPAE@Z 1000114b f   endian.obj
 0001:0000015e       ?set_java@Endian@@SAXPAEG@Z 1000115e f   endian.obj
 0001:00000171       ?decompress@ZipDecompressor@@SAEPAX_K01PAPAD@Z 10001171 f   imageDecompressor.obj
 0001:00000194       ?decompress_int@SharedStringDecompressor@@CAHAAPAE@Z 10001194 f   imageDecompressor.obj
 0001:0000020e       ?decompress_resource@ImageDecompressor@@SAXPAE0_KPBVImageStrings@@PAVEndian@@@Z 1000120e f   imageDecompressor.obj
 0001:00000321       ?decompress_resource@SharedStringDecompressor@@UAEXPAE0PAUResourceHeader@@PBVImageStrings@@@Z 10001321 f   imageDecompressor.obj
 0001:000005b5       ?decompress_resource@ZipDecompressor@@UAEXPAE0PAUResourceHeader@@PBVImageStrings@@@Z 100015b5 f   imageDecompressor.obj
 0001:000005e2       ?getU4@ImageDecompressor@@CAIPAEPAVEndian@@@Z 100015e2 f   imageDecompressor.obj
 0001:00000605       ?getU8@ImageDecompressor@@CA_KPAEPAVEndian@@@Z 10001605 f   imageDecompressor.obj
 0001:0000066c       ?get_decompressor@ImageDecompressor@@SAPAV1@PBD@Z 1000166c f   imageDecompressor.obj
 0001:000006a9       ?image_decompressor_init@ImageDecompressor@@SAXXZ 100016a9 f   imageDecompressor.obj
 0001:00000749       ___local_stdio_printf_options 10001749 f i imageDecompressor.obj
 0001:0000074f       __vfprintf_l               1000174f f i imageDecompressor.obj
 0001:00000773       _printf                    10001773 f i imageDecompressor.obj
 0001:00000791       ??0ImageFileReader@@AAE@PBD_N@Z 10001791 f   imageFile.obj
 0001:000007d7       ??0ImageFileReaderTable@@QAE@XZ 100017d7 f   imageFile.obj
 0001:000007f5       ??1ImageFileReader@@AAE@XZ 100017f5 f   imageFile.obj
 0001:00000821       ?add@ImageFileReaderTable@@QAEXPAVImageFileReader@@@Z 10001821 f   imageFile.obj
 0001:00000857       ?attribute_value@ImageLocation@@CA_KPAEE@Z 10001857 f i imageFile.obj
 0001:00000898       ?clear_data@ImageLocation@@QAEXXZ 10001898 f   imageFile.obj
 0001:000008a6       ?close@ImageFileReader@@QAEXXZ 100018a6 f   imageFile.obj
 0001:000008ee       ?close@ImageFileReader@@SAXPAV1@@Z 100018ee f   imageFile.obj
 0001:0000092b       ?find@ImageStrings@@SAHPAVEndian@@PBDPAHI@Z 1000192b f   imageFile.obj
 0001:0000097f       ?find_image@ImageFileReader@@SAPAV1@PBD@Z 1000197f f   imageFile.obj
 0001:000009ce       ?find_location@ImageFileReader@@QBE_NPBDAAVImageLocation@@@Z 100019ce f   imageFile.obj
 0001:00000a1d       ?find_location_index@ImageFileReader@@QBEIPBDPA_K@Z 10001a1d f   imageFile.obj
 0001:00000ad4       ?get_image_module_data@ImageFileReader@@QAEPAVImageModuleData@@XZ 10001ad4 f   imageFile.obj
 0001:00000ad8       ?get_location_data@ImageFileReader@@QBEPAEI@Z 10001ad8 f i imageFile.obj
 0001:00000b02       ?get_resource@ImageFileReader@@QBEXAAVImageLocation@@PAE@Z 10001b02 f   imageFile.obj
 0001:00000bcc       ?get_resource@ImageFileReader@@QBEXIPAE@Z 10001bcc f   imageFile.obj
 0001:00000c2a       ?get_strings@ImageFileReader@@QBE?BVImageStrings@@XZ 10001c2a f i imageFile.obj
 0001:00000c4a       ?hash_code@ImageStrings@@SAHPBDH@Z 10001c4a f   imageFile.obj
 0001:00000c76       ?index_size@ImageFileReader@@AAEIXZ 10001c76 f i imageFile.obj
 0001:00000cac       ?open@ImageFileReader@@QAE_NXZ 10001cac f   imageFile.obj
 0001:00000de8       ?open@ImageFileReader@@SAPAV1@PBD_N@Z 10001de8 f   imageFile.obj
 0001:00000eba       ?package_to_module@ImageModuleData@@QAEPBDPBD@Z 10001eba f   imageFile.obj
 0001:0000101a       ?read_at@ImageFileReader@@QBE_NPAE_K1@Z 1000201a f   imageFile.obj
 0001:0000104b       ?remove@ImageFileReaderTable@@QAEXPAVImageFileReader@@@Z 1000204b f   imageFile.obj
 0001:0000109c       ?set_data@ImageLocation@@QAEXPAE@Z 1000209c f   imageFile.obj
 0001:000010e5       ?starts_with@ImageStrings@@SAPBDPBD0@Z 100020e5 f   imageFile.obj
 0001:0000110e       ?verify_location@ImageFileReader@@QBE_NAAVImageLocation@@PBD@Z 1000210e f   imageFile.obj
 0001:000011af       _JIMAGE_Close              100021af f   jimage.obj
 0001:000011b4       _JIMAGE_FindResource       100021b4 f   jimage.obj
 0001:00001283       _JIMAGE_GetResource        10002283 f   jimage.obj
 0001:0000129c       _JIMAGE_Open               1000229c f   jimage.obj
 0001:000012b1       _JIMAGE_PackageToModule    100022b1 f   jimage.obj
 0001:000012c6       _JIMAGE_ResourceIterator   100022c6 f   jimage.obj
 0001:000013a6       ??0SimpleCriticalSection@@QAE@XZ 100023a6 f   osSupport_windows.obj
 0001:000013b4       ?close@osSupport@@SAJJ@Z   100023b4 f   osSupport_windows.obj
 0001:000013ba       ?enter@SimpleCriticalSection@@AAEXXZ 100023ba f   osSupport_windows.obj
 0001:000013c2       ?exit@SimpleCriticalSection@@AAEXXZ 100023c2 f   osSupport_windows.obj
 0001:000013ca       ?map_memory@osSupport@@SAPAXJPBDII@Z 100023ca f   osSupport_windows.obj
 0001:0000142b       ?openReadOnly@osSupport@@SAJPBD@Z 1000242b f   osSupport_windows.obj
 0001:00001440       ?read@osSupport@@SA_JJPAD_J1@Z 10002440 f   osSupport_windows.obj
 0001:0000148e       ?size@osSupport@@SA_JPBD@Z 1000248e f   osSupport_windows.obj
 0001:000014d2       ?unmap_memory@osSupport@@SAHPAXI@Z 100024d2 f   osSupport_windows.obj
 0001:000014dd       ??_Etype_info@@UAEPAXI@Z   100024dd f i MSVCRT:std_type_info_static.obj
 0001:000014dd       ??_Gtype_info@@UAEPAXI@Z   100024dd f i MSVCRT:std_type_info_static.obj
 0001:00001500       ??2@YAPAXI@Z               10002500 f   MSVCRT:new_scalar.obj
 0001:00001530       ??_U@YAPAXI@Z              10002530 f   MSVCRT:new_array.obj
 0001:00001539       ??_V@YAXPAX@Z              10002539 f   MSVCRT:delete_array.obj
 0001:0000153e       @__security_check_cookie@4 1000253e f   MSVCRT:secchk.obj
 0001:0000154c       ??3@YAXPAXI@Z              1000254c f   MSVCRT:delete_scalar_size.obj
 0001:0000155a       ___raise_securityfailure   1000255a f   MSVCRT:gs_report.obj
 0001:00001582       ___report_gsfailure        10002582 f   MSVCRT:gs_report.obj
 0001:0000167c       ___report_rangecheckfailure 1000267c f   MSVCRT:gs_report.obj
 0001:00001688       ___report_securityfailure  10002688 f   MSVCRT:gs_report.obj
 0001:00001760       __alloca_probe             10002760 f   MSVCRT:chkstk.obj
 0001:00001760       __chkstk                   10002760 f   MSVCRT:chkstk.obj
 0001:00001acb       __DllMainCRTStartup@12     10002acb f   MSVCRT:dll_dllmain.obj
 0001:00001aee       ??0bad_alloc@std@@QAE@ABV01@@Z 10002aee f i MSVCRT:throw_bad_alloc.obj
 0001:00001b09       ??0bad_alloc@std@@QAE@XZ   10002b09 f i MSVCRT:throw_bad_alloc.obj
 0001:00001b21       ??0bad_array_new_length@std@@QAE@ABV01@@Z 10002b21 f i MSVCRT:throw_bad_alloc.obj
 0001:00001b3c       ??0bad_array_new_length@std@@QAE@XZ 10002b3c f i MSVCRT:throw_bad_alloc.obj
 0001:00001b54       ??0exception@std@@QAE@ABV01@@Z 10002b54 f i MSVCRT:throw_bad_alloc.obj
 0001:00001b80       ??1bad_alloc@std@@UAE@XZ   10002b80 f i MSVCRT:throw_bad_alloc.obj
 0001:00001b80       ??1bad_array_new_length@std@@UAE@XZ 10002b80 f i MSVCRT:throw_bad_alloc.obj
 0001:00001b91       ??_Ebad_alloc@std@@UAEPAXI@Z 10002b91 f i MSVCRT:throw_bad_alloc.obj
 0001:00001b91       ??_Ebad_array_new_length@std@@UAEPAXI@Z 10002b91 f i MSVCRT:throw_bad_alloc.obj
 0001:00001b91       ??_Eexception@std@@UAEPAXI@Z 10002b91 f i MSVCRT:throw_bad_alloc.obj
 0001:00001b91       ??_Gbad_alloc@std@@UAEPAXI@Z 10002b91 f i MSVCRT:throw_bad_alloc.obj
 0001:00001b91       ??_Gbad_array_new_length@std@@UAEPAXI@Z 10002b91 f i MSVCRT:throw_bad_alloc.obj
 0001:00001b91       ??_Gexception@std@@UAEPAXI@Z 10002b91 f i MSVCRT:throw_bad_alloc.obj
 0001:00001bbe       ?__scrt_throw_std_bad_alloc@@YAXXZ 10002bbe f   MSVCRT:throw_bad_alloc.obj
 0001:00001bdb       ?__scrt_throw_std_bad_array_new_length@@YAXXZ 10002bdb f   MSVCRT:throw_bad_alloc.obj
 0001:00001bf8       ?what@exception@std@@UBEPBDXZ 10002bf8 f i MSVCRT:throw_bad_alloc.obj
 0001:00001c05       ??3@YAXPAX@Z               10002c05 f   MSVCRT:delete_scalar.obj
 0001:00001c57       ___security_init_cookie    10002c57 f   MSVCRT:gs_support.obj
 0001:00001ca2       _DllMain@12                10002ca2 f   MSVCRT:dll_dllmain_stub.obj
 0001:00001cc4       ?__scrt_initialize_type_info@@YAXXZ 10002cc4 f   MSVCRT:tncleanup.obj
 0001:00001cd0       ?__scrt_uninitialize_type_info@@YAXXZ 10002cd0 f   MSVCRT:tncleanup.obj
 0001:00001cdc       ___local_stdio_scanf_options 10002cdc f i MSVCRT:default_local_stdio_options.obj
 0001:00001ce2       ___scrt_initialize_default_local_stdio_options 10002ce2 f   MSVCRT:default_local_stdio_options.obj
 0001:00001d43       ___scrt_acquire_startup_lock 10002d43 f   MSVCRT:utility.obj
 0001:00001d75       ___scrt_dllmain_after_initialize_c 10002d75 f   MSVCRT:utility.obj
 0001:00001da0       ___scrt_dllmain_before_initialize_c 10002da0 f   MSVCRT:utility.obj
 0001:00001dae       ___scrt_dllmain_crt_thread_attach 10002dae f   MSVCRT:utility.obj
 0001:00001dcd       ___scrt_dllmain_crt_thread_detach 10002dcd f   MSVCRT:utility.obj
 0001:00001dda       ___scrt_dllmain_exception_filter 10002dda f   MSVCRT:utility.obj
 0001:00001e0e       ___scrt_dllmain_uninitialize_c 10002e0e f   MSVCRT:utility.obj
 0001:00001e31       ___scrt_dllmain_uninitialize_critical 10002e31 f   MSVCRT:utility.obj
 0001:00001e3e       ___scrt_initialize_crt     10002e3e f   MSVCRT:utility.obj
 0001:00001e77       ___scrt_initialize_onexit_tables 10002e77 f   MSVCRT:utility.obj
 0001:00001efe       ___scrt_is_nonwritable_in_current_image 10002efe f   MSVCRT:utility.obj
 0001:00001f92       ___scrt_release_startup_lock 10002f92 f   MSVCRT:utility.obj
 0001:00001faf       ___scrt_uninitialize_crt   10002faf f   MSVCRT:utility.obj
 0001:00001fd7       ___scrt_get_dyn_tls_init_callback 10002fd7 f   MSVCRT:dyn_tls_init.obj
 0001:00001fdd       ___scrt_fastfail           10002fdd f   MSVCRT:utility_desktop.obj
 0001:000020f8       __crt_debugger_hook        100030f8 f   MSVCRT:utility_desktop.obj
 0001:00002100       __RTC_Initialize           10003100 f   MSVCRT:initsect.obj
 0001:0000212c       __RTC_Terminate            1000312c f   MSVCRT:initsect.obj
 0001:00002160       __SEH_prolog4              10003160 f   MSVCRT:sehprolg4.obj
 0001:000021a5       __except_handler4          100031a5 f   MSVCRT:chandler4gs.obj
 0001:000021d4       @_guard_check_icall_nop@4  100031d4 f i MSVCRT:guard_support.obj
 0001:000021d7       ___isa_available_init      100031d7 f   MSVCRT:cpu_disp.obj
 0001:000023ab       __get_startup_argv_mode    100033ab f   MSVCRT:argv_mode.obj
 0001:000023af       ___scrt_is_ucrt_dll_in_use 100033af f   MSVCRT:ucrt_detection.obj
 0001:000023bb       _memcpy                    100033bb f   vcruntime:VCRUNTIME140.dll
 0001:000023c1       _memset                    100033c1 f   vcruntime:VCRUNTIME140.dll
 0001:000023c7       ___std_exception_copy      100033c7 f   vcruntime:VCRUNTIME140.dll
 0001:000023cd       ___std_exception_destroy   100033cd f   vcruntime:VCRUNTIME140.dll
 0001:000023d3       __CxxThrowException@8      100033d3 f   vcruntime:VCRUNTIME140.dll
 0001:000023d9       ___std_type_info_destroy_list 100033d9 f   vcruntime:VCRUNTIME140.dll
 0001:000023df       __except_handler4_common   100033df f   vcruntime:VCRUNTIME140.dll
 0001:000023e5       _strcmp                    100033e5 f   ucrt:api-ms-win-crt-string-l1-1-0.dll
 0001:000023eb       _strlen                    100033eb f   ucrt:api-ms-win-crt-string-l1-1-0.dll
 0001:000023f1       _strcat                    100033f1 f   ucrt:api-ms-win-crt-string-l1-1-0.dll
 0001:000023f7       _strcpy                    100033f7 f   ucrt:api-ms-win-crt-string-l1-1-0.dll
 0001:000023fd       __callnewh                 100033fd f   ucrt:api-ms-win-crt-heap-l1-1-0.dll
 0001:00002403       _malloc                    10003403 f   ucrt:api-ms-win-crt-heap-l1-1-0.dll
 0001:00002409       __initterm                 10003409 f   ucrt:api-ms-win-crt-runtime-l1-1-0.dll
 0001:0000240f       __initterm_e               1000340f f   ucrt:api-ms-win-crt-runtime-l1-1-0.dll
 0001:00002415       _free                      10003415 f   ucrt:api-ms-win-crt-heap-l1-1-0.dll
 0001:0000241b       __seh_filter_dll           1000341b f   ucrt:api-ms-win-crt-runtime-l1-1-0.dll
 0001:00002421       __configure_narrow_argv    10003421 f   ucrt:api-ms-win-crt-runtime-l1-1-0.dll
 0001:00002427       __initialize_narrow_environment 10003427 f   ucrt:api-ms-win-crt-runtime-l1-1-0.dll
 0001:0000242d       __initialize_onexit_table  1000342d f   ucrt:api-ms-win-crt-runtime-l1-1-0.dll
 0001:00002433       __execute_onexit_table     10003433 f   ucrt:api-ms-win-crt-runtime-l1-1-0.dll
 0001:00002439       __cexit                    10003439 f   ucrt:api-ms-win-crt-runtime-l1-1-0.dll
 0001:0000243f       ___acrt_initialize         1000343f f   MSVCRT:ucrt_stubs.obj
 0001:0000243f       ___acrt_thread_attach      1000343f f   MSVCRT:ucrt_stubs.obj
 0001:0000243f       ___acrt_thread_detach      1000343f f   MSVCRT:ucrt_stubs.obj
 0001:0000243f       ___acrt_uninitialize       1000343f f   MSVCRT:ucrt_stubs.obj
 0001:0000243f       ___acrt_uninitialize_critical 1000343f f   MSVCRT:ucrt_stubs.obj
 0001:0000243f       ___scrt_stub_for_acrt_initialize 1000343f f   MSVCRT:ucrt_stubs.obj
 0001:0000243f       ___scrt_stub_for_acrt_thread_attach 1000343f f   MSVCRT:ucrt_stubs.obj
 0001:0000243f       ___scrt_stub_for_acrt_thread_detach 1000343f f   MSVCRT:ucrt_stubs.obj
 0001:0000243f       ___scrt_stub_for_acrt_uninitialize 1000343f f   MSVCRT:ucrt_stubs.obj
 0001:0000243f       ___scrt_stub_for_acrt_uninitialize_critical 1000343f f   MSVCRT:ucrt_stubs.obj
 0001:0000243f       ___vcrt_initialize         1000343f f   MSVCRT:ucrt_stubs.obj
 0001:0000243f       ___vcrt_thread_attach      1000343f f   MSVCRT:ucrt_stubs.obj
 0001:0000243f       ___vcrt_thread_detach      1000343f f   MSVCRT:ucrt_stubs.obj
 0001:0000243f       ___vcrt_uninitialize       1000343f f   MSVCRT:ucrt_stubs.obj
 0001:0000243f       ___vcrt_uninitialize_critical 1000343f f   MSVCRT:ucrt_stubs.obj
 0001:00002442       ___scrt_stub_for_is_c_termination_complete 10003442 f   MSVCRT:ucrt_stubs.obj
 0001:00002442       __is_c_termination_complete 10003442 f   MSVCRT:ucrt_stubs.obj
 0001:00002445       __filter_x86_sse2_floating_point_exception 10003445 f   MSVCRT:x86_exception_filter.obj
 0001:00002445       __filter_x86_sse2_floating_point_exception_default 10003445 f   MSVCRT:x86_exception_filter.obj
 0002:00000000       __imp__GetModuleHandleA@4  10004000     kernel32:KERNEL32.dll
 0002:00000004       __imp__GetProcAddress@8    10004004     kernel32:KERNEL32.dll
 0002:00000008       __imp__LoadLibraryA@4      10004008     kernel32:KERNEL32.dll
 0002:0000000c       __imp__CreateFileA@28      1000400c     kernel32:KERNEL32.dll
 0002:00000010       __imp__ReadFile@20         10004010     kernel32:KERNEL32.dll
 0002:00000014       __imp__CloseHandle@4       10004014     kernel32:KERNEL32.dll
 0002:00000018       __imp__InitializeCriticalSection@4 10004018     kernel32:KERNEL32.dll
 0002:0000001c       __imp__EnterCriticalSection@4 1000401c     kernel32:KERNEL32.dll
 0002:00000020       __imp__LeaveCriticalSection@4 10004020     kernel32:KERNEL32.dll
 0002:00000024       __imp__MapViewOfFileEx@24  10004024     kernel32:KERNEL32.dll
 0002:00000028       __imp__UnmapViewOfFile@4   10004028     kernel32:KERNEL32.dll
 0002:0000002c       __imp__CreateFileMappingA@24 1000402c     kernel32:KERNEL32.dll
 0002:00000030       __imp__UnhandledExceptionFilter@4 10004030     kernel32:KERNEL32.dll
 0002:00000034       __imp__SetUnhandledExceptionFilter@4 10004034     kernel32:KERNEL32.dll
 0002:00000038       __imp__GetCurrentProcess@0 10004038     kernel32:KERNEL32.dll
 0002:0000003c       __imp__TerminateProcess@8  1000403c     kernel32:KERNEL32.dll
 0002:00000040       __imp__IsProcessorFeaturePresent@4 10004040     kernel32:KERNEL32.dll
 0002:00000044       __imp__QueryPerformanceCounter@4 10004044     kernel32:KERNEL32.dll
 0002:00000048       __imp__GetCurrentProcessId@0 10004048     kernel32:KERNEL32.dll
 0002:0000004c       __imp__GetCurrentThreadId@0 1000404c     kernel32:KERNEL32.dll
 0002:00000050       __imp__GetSystemTimeAsFileTime@4 10004050     kernel32:KERNEL32.dll
 0002:00000054       __imp__DisableThreadLibraryCalls@4 10004054     kernel32:KERNEL32.dll
 0002:00000058       __imp__InitializeSListHead@4 10004058     kernel32:KERNEL32.dll
 0002:0000005c       __imp__IsDebuggerPresent@0 1000405c     kernel32:KERNEL32.dll
 0002:00000060       \177KERNEL32_NULL_THUNK_DATA 10004060     kernel32:KERNEL32.dll
 0002:00000064       __imp__memcpy              10004064     vcruntime:VCRUNTIME140.dll
 0002:00000068       __imp__memset              10004068     vcruntime:VCRUNTIME140.dll
 0002:0000006c       __imp____std_exception_copy 1000406c     vcruntime:VCRUNTIME140.dll
 0002:00000070       __imp____std_exception_destroy 10004070     vcruntime:VCRUNTIME140.dll
 0002:00000074       __imp___CxxThrowException@8 10004074     vcruntime:VCRUNTIME140.dll
 0002:00000078       __imp____std_type_info_destroy_list 10004078     vcruntime:VCRUNTIME140.dll
 0002:0000007c       __imp___except_handler4_common 1000407c     vcruntime:VCRUNTIME140.dll
 0002:00000080       \177VCRUNTIME140_NULL_THUNK_DATA 10004080     vcruntime:VCRUNTIME140.dll
 0002:00000084       __imp___stat64i32          10004084     ucrt:api-ms-win-crt-filesystem-l1-1-0.dll
 0002:00000088       \177api-ms-win-crt-filesystem-l1-1-0_NULL_THUNK_DATA 10004088     ucrt:api-ms-win-crt-filesystem-l1-1-0.dll
 0002:0000008c       __imp___callnewh           1000408c     ucrt:api-ms-win-crt-heap-l1-1-0.dll
 0002:00000090       __imp__malloc              10004090     ucrt:api-ms-win-crt-heap-l1-1-0.dll
 0002:00000094       __imp__realloc             10004094     ucrt:api-ms-win-crt-heap-l1-1-0.dll
 0002:00000098       __imp__calloc              10004098     ucrt:api-ms-win-crt-heap-l1-1-0.dll
 0002:0000009c       __imp__free                1000409c     ucrt:api-ms-win-crt-heap-l1-1-0.dll
 0002:000000a0       \177api-ms-win-crt-heap-l1-1-0_NULL_THUNK_DATA 100040a0     ucrt:api-ms-win-crt-heap-l1-1-0.dll
 0002:000000a4       __imp___cexit              100040a4     ucrt:api-ms-win-crt-runtime-l1-1-0.dll
 0002:000000a8       __imp___initterm           100040a8     ucrt:api-ms-win-crt-runtime-l1-1-0.dll
 0002:000000ac       __imp___initterm_e         100040ac     ucrt:api-ms-win-crt-runtime-l1-1-0.dll
 0002:000000b0       __imp___execute_onexit_table 100040b0     ucrt:api-ms-win-crt-runtime-l1-1-0.dll
 0002:000000b4       __imp___seh_filter_dll     100040b4     ucrt:api-ms-win-crt-runtime-l1-1-0.dll
 0002:000000b8       __imp___configure_narrow_argv 100040b8     ucrt:api-ms-win-crt-runtime-l1-1-0.dll
 0002:000000bc       __imp___initialize_narrow_environment 100040bc     ucrt:api-ms-win-crt-runtime-l1-1-0.dll
 0002:000000c0       __imp___initialize_onexit_table 100040c0     ucrt:api-ms-win-crt-runtime-l1-1-0.dll
 0002:000000c4       \177api-ms-win-crt-runtime-l1-1-0_NULL_THUNK_DATA 100040c4     ucrt:api-ms-win-crt-runtime-l1-1-0.dll
 0002:000000c8       __imp____acrt_iob_func     100040c8     ucrt:api-ms-win-crt-stdio-l1-1-0.dll
 0002:000000cc       __imp____stdio_common_vfprintf 100040cc     ucrt:api-ms-win-crt-stdio-l1-1-0.dll
 0002:000000d0       __imp___open               100040d0     ucrt:api-ms-win-crt-stdio-l1-1-0.dll
 0002:000000d0       __imp__open                100040d0     ucrt:api-ms-win-crt-stdio-l1-1-0.dll
 0002:000000d4       __imp___close              100040d4     ucrt:api-ms-win-crt-stdio-l1-1-0.dll
 0002:000000d4       __imp__close               100040d4     ucrt:api-ms-win-crt-stdio-l1-1-0.dll
 0002:000000d8       __imp___get_osfhandle      100040d8     ucrt:api-ms-win-crt-stdio-l1-1-0.dll
 0002:000000dc       \177api-ms-win-crt-stdio-l1-1-0_NULL_THUNK_DATA 100040dc     ucrt:api-ms-win-crt-stdio-l1-1-0.dll
 0002:000000e0       __imp__strcat              100040e0     ucrt:api-ms-win-crt-string-l1-1-0.dll
 0002:000000e4       __imp__strlen              100040e4     ucrt:api-ms-win-crt-string-l1-1-0.dll
 0002:000000e8       __imp__strcpy              100040e8     ucrt:api-ms-win-crt-string-l1-1-0.dll
 0002:000000ec       __imp__strncpy             100040ec     ucrt:api-ms-win-crt-string-l1-1-0.dll
 0002:000000f0       __imp__strcmp              100040f0     ucrt:api-ms-win-crt-string-l1-1-0.dll
 0002:000000f4       \177api-ms-win-crt-string-l1-1-0_NULL_THUNK_DATA 100040f4     ucrt:api-ms-win-crt-string-l1-1-0.dll
 0002:000000f8       ___guard_check_icall_fptr  100040f8     MSVCRT:guard_support.obj
 0002:000000fc       ___castguard_check_failure_os_handled_fptr 100040fc     MSVCRT:guard_support.obj
 0002:00000100       ___xc_a                    10004100     MSVCRT:initializers.obj
 0002:0000010c       ___xc_z                    1000410c     MSVCRT:initializers.obj
 0002:00000110       ___xi_a                    10004110     MSVCRT:initializers.obj
 0002:00000114       ___xi_z                    10004114     MSVCRT:initializers.obj
 0002:00000118       ___xp_a                    10004118     MSVCRT:initializers.obj
 0002:0000011c       ___xp_z                    1000411c     MSVCRT:initializers.obj
 0002:00000120       ___xt_a                    10004120     MSVCRT:initializers.obj
 0002:00000124       ___xt_z                    10004124     MSVCRT:initializers.obj
 0002:0000012c       ??_7NativeEndian@@6B@      1000412c     endian.obj
 0002:00000160       ??_7SwappingEndian@@6B@    10004160     endian.obj
 0002:00000190       ?sizes@SharedStringDecompressor@@0QBEB 10004190     imageDecompressor.obj
 0002:000001a8       ??_7ZipDecompressor@@6B@   100041a8     imageDecompressor.obj
 0002:000001b0       ??_7SharedStringDecompressor@@6B@ 100041b0     imageDecompressor.obj
 0002:000001b4       ??_C@_07PAHBEOOH@zip?4dll@ 100041b4     imageDecompressor.obj
 0002:000001bc       ??_C@_0BB@FGJGIFHO@ZIP_InflateFully@ 100041bc     imageDecompressor.obj
 0002:000001d0       ??_C@_03LCAAOJEC@zip@      100041d0     imageDecompressor.obj
 0002:000001d4       ??_C@_0L@OENLBBHC@compact?9cp@ 100041d4     imageDecompressor.obj
 0002:000001e0       ??_C@_0CK@CHFPEALO@Failure?0?5expecting?5?$CFllu?5but?5get@ 100041e0     imageDecompressor.obj
 0002:0000020c       ??_C@_0L@ELHBAEMN@?1packages?1@ 1000420c     imageFile.obj
 0002:00000218       ??_C@_07DFGEOAEG@modules@  10004218     jimage.obj
 0002:00000220       ??_C@_08GFNEJDPJ@packages@ 10004220     jimage.obj
 0002:0000022c       ??_C@_01LAKCGALK@9@        1000422c     jimage.obj
 0002:00000234       ??_7type_info@@6B@         10004234     MSVCRT:std_type_info_static.obj
 0002:00000240       __pDefaultRawDllMain       10004240     MSVCRT:dll_dllmain.obj
 0002:00000240       __pRawDllMain              10004240     MSVCRT:dll_dllmain.obj
 0002:00000248       ??_7exception@std@@6B@     10004248     MSVCRT:throw_bad_alloc.obj
 0002:00000250       ??_C@_0BC@EOODALEL@Unknown?5exception@ 10004250     MSVCRT:throw_bad_alloc.obj
 0002:00000268       ??_7bad_alloc@std@@6B@     10004268     MSVCRT:throw_bad_alloc.obj
 0002:00000270       ??_C@_0P@GHFPNOJB@bad?5allocation@ 10004270     MSVCRT:throw_bad_alloc.obj
 0002:00000284       ??_7bad_array_new_length@std@@6B@ 10004284     MSVCRT:throw_bad_alloc.obj
 0002:0000028c       ??_C@_0BF@KINCDENJ@bad?5array?5new?5length@ 1000428c     MSVCRT:throw_bad_alloc.obj
 0002:000002a8       __load_config_used         100042a8     MSVCRT:loadcfg.obj
 0002:00000400       ??_R3Endian@@8             10004400     endian.obj
 0002:00000410       ??_R2Endian@@8             10004410     endian.obj
 0002:00000418       ??_R1A@?0A@EA@Endian@@8    10004418     endian.obj
 0002:00000434       ??_R4NativeEndian@@6B@     10004434     endian.obj
 0002:00000448       ??_R3NativeEndian@@8       10004448     endian.obj
 0002:00000458       ??_R2NativeEndian@@8       10004458     endian.obj
 0002:00000464       ??_R1A@?0A@EA@NativeEndian@@8 10004464     endian.obj
 0002:00000480       ??_R4SwappingEndian@@6B@   10004480     endian.obj
 0002:00000494       ??_R3SwappingEndian@@8     10004494     endian.obj
 0002:000004a4       ??_R2SwappingEndian@@8     100044a4     endian.obj
 0002:000004b0       ??_R1A@?0A@EA@SwappingEndian@@8 100044b0     endian.obj
 0002:000004cc       ??_R3ImageDecompressor@@8  100044cc     imageDecompressor.obj
 0002:000004dc       ??_R2ImageDecompressor@@8  100044dc     imageDecompressor.obj
 0002:000004e4       ??_R1A@?0A@EA@ImageDecompressor@@8 100044e4     imageDecompressor.obj
 0002:00000500       ??_R4ZipDecompressor@@6B@  10004500     imageDecompressor.obj
 0002:00000514       ??_R3ZipDecompressor@@8    10004514     imageDecompressor.obj
 0002:00000524       ??_R2ZipDecompressor@@8    10004524     imageDecompressor.obj
 0002:00000530       ??_R1A@?0A@EA@ZipDecompressor@@8 10004530     imageDecompressor.obj
 0002:0000054c       ??_R4SharedStringDecompressor@@6B@ 1000454c     imageDecompressor.obj
 0002:00000560       ??_R3SharedStringDecompressor@@8 10004560     imageDecompressor.obj
 0002:00000570       ??_R2SharedStringDecompressor@@8 10004570     imageDecompressor.obj
 0002:0000057c       ??_R1A@?0A@EA@SharedStringDecompressor@@8 1000457c     imageDecompressor.obj
 0002:00000598       ??_R4type_info@@6B@        10004598     MSVCRT:std_type_info_static.obj
 0002:000005ac       ??_R3type_info@@8          100045ac     MSVCRT:std_type_info_static.obj
 0002:000005bc       ??_R2type_info@@8          100045bc     MSVCRT:std_type_info_static.obj
 0002:000005c4       ??_R1A@?0A@EA@type_info@@8 100045c4     MSVCRT:std_type_info_static.obj
 0002:000005e0       ??_R4exception@std@@6B@    100045e0     MSVCRT:throw_bad_alloc.obj
 0002:000005f4       ??_R3exception@std@@8      100045f4     MSVCRT:throw_bad_alloc.obj
 0002:00000604       ??_R2exception@std@@8      10004604     MSVCRT:throw_bad_alloc.obj
 0002:0000060c       ??_R1A@?0A@EA@exception@std@@8 1000460c     MSVCRT:throw_bad_alloc.obj
 0002:00000628       ??_R4bad_alloc@std@@6B@    10004628     MSVCRT:throw_bad_alloc.obj
 0002:0000063c       ??_R3bad_alloc@std@@8      1000463c     MSVCRT:throw_bad_alloc.obj
 0002:0000064c       ??_R2bad_alloc@std@@8      1000464c     MSVCRT:throw_bad_alloc.obj
 0002:00000658       ??_R1A@?0A@EA@bad_alloc@std@@8 10004658     MSVCRT:throw_bad_alloc.obj
 0002:00000674       ??_R4bad_array_new_length@std@@6B@ 10004674     MSVCRT:throw_bad_alloc.obj
 0002:00000688       ??_R3bad_array_new_length@std@@8 10004688     MSVCRT:throw_bad_alloc.obj
 0002:00000698       ??_R2bad_array_new_length@std@@8 10004698     MSVCRT:throw_bad_alloc.obj
 0002:000006a8       ??_R1A@?0A@EA@bad_array_new_length@std@@8 100046a8     MSVCRT:throw_bad_alloc.obj
 0002:000006c4       ___safe_se_handler_table   100046c4     <linker-defined>
 0002:000006c8       ___volatile_metadata       100046c8     <linker-defined>
 0002:00000a28       ___rtc_iaa                 10004a28     MSVCRT:initsect.obj
 0002:00000a2c       ___rtc_izz                 10004a2c     MSVCRT:initsect.obj
 0002:00000a30       ___rtc_taa                 10004a30     MSVCRT:initsect.obj
 0002:00000a34       ___rtc_tzz                 10004a34     MSVCRT:initsect.obj
 0002:00000a9c       __TI2?AVbad_alloc@std@@    10004a9c     MSVCRT:throw_bad_alloc.obj
 0002:00000aac       __CTA2?AVbad_alloc@std@@   10004aac     MSVCRT:throw_bad_alloc.obj
 0002:00000ab8       __CT??_R0?AVbad_alloc@std@@@8??0bad_alloc@std@@QAE@ABV01@@Z12 10004ab8     MSVCRT:throw_bad_alloc.obj
 0002:00000ad4       __CT??_R0?AVexception@std@@@8??0exception@std@@QAE@ABV01@@Z12 10004ad4     MSVCRT:throw_bad_alloc.obj
 0002:00000af0       __TI3?AVbad_array_new_length@std@@ 10004af0     MSVCRT:throw_bad_alloc.obj
 0002:00000b00       __CTA3?AVbad_array_new_length@std@@ 10004b00     MSVCRT:throw_bad_alloc.obj
 0002:00000b10       __CT??_R0?AVbad_array_new_length@std@@@8??0bad_array_new_length@std@@QAE@ABV01@@Z12 10004b10     MSVCRT:throw_bad_alloc.obj
 0002:00000c74       __IMPORT_DESCRIPTOR_KERNEL32 10004c74     kernel32:KERNEL32.dll
 0002:00000c88       __IMPORT_DESCRIPTOR_VCRUNTIME140 10004c88     vcruntime:VCRUNTIME140.dll
 0002:00000c9c       __IMPORT_DESCRIPTOR_api-ms-win-crt-stdio-l1-1-0 10004c9c     ucrt:api-ms-win-crt-stdio-l1-1-0.dll
 0002:00000cb0       __IMPORT_DESCRIPTOR_api-ms-win-crt-string-l1-1-0 10004cb0     ucrt:api-ms-win-crt-string-l1-1-0.dll
 0002:00000cc4       __IMPORT_DESCRIPTOR_api-ms-win-crt-heap-l1-1-0 10004cc4     ucrt:api-ms-win-crt-heap-l1-1-0.dll
 0002:00000cd8       __IMPORT_DESCRIPTOR_api-ms-win-crt-filesystem-l1-1-0 10004cd8     ucrt:api-ms-win-crt-filesystem-l1-1-0.dll
 0002:00000cec       __IMPORT_DESCRIPTOR_api-ms-win-crt-runtime-l1-1-0 10004cec     ucrt:api-ms-win-crt-runtime-l1-1-0.dll
 0002:00000d00       __NULL_IMPORT_DESCRIPTOR   10004d00     kernel32:KERNEL32.dll
 0003:00000000       ?_native@NativeEndian@@0V1@A 10006000     endian.obj
 0003:00000004       ?_swapping@SwappingEndian@@0V1@A 10006004     endian.obj
 0003:00000008       ___security_cookie_complement 10006008     MSVCRT:gs_cookie.obj
 0003:0000000c       ___security_cookie         1000600c     MSVCRT:gs_cookie.obj
 0003:00000010       ___scrt_native_dllmain_reason 10006010     MSVCRT:utility.obj
 0003:00000020       ___isa_enabled             10006020     MSVCRT:cpu_disp.obj
 0003:00000024       ___scrt_ucrt_dll_is_in_use 10006024     MSVCRT:ucrt_stubs.obj
 0003:00000028       ??_R0?AVbad_alloc@std@@@8  10006028     MSVCRT:throw_bad_alloc.obj
 0003:00000044       ??_R0?AVexception@std@@@8  10006044     MSVCRT:throw_bad_alloc.obj
 0003:00000060       ??_R0?AVbad_array_new_length@std@@@8 10006060     MSVCRT:throw_bad_alloc.obj
 0003:00000088       ??_R0?AVEndian@@@8         10006088     endian.obj
 0003:000000a0       ??_R0?AVNativeEndian@@@8   100060a0     endian.obj
 0003:000000bc       ??_R0?AVSwappingEndian@@@8 100060bc     endian.obj
 0003:000000dc       ??_R0?AVImageDecompressor@@@8 100060dc     imageDecompressor.obj
 0003:000000fc       ??_R0?AVZipDecompressor@@@8 100060fc     imageDecompressor.obj
 0003:0000011c       ??_R0?AVSharedStringDecompressor@@@8 1000611c     imageDecompressor.obj
 0003:00000144       ??_R0?AVtype_info@@@8      10006144     MSVCRT:std_type_info_static.obj
 0003:00000160       ?_decompressors@ImageDecompressor@@0PAPAV1@A 10006160     imageDecompressor.obj
 0003:00000164       ?_decompressors_num@ImageDecompressor@@0HA 10006164     imageDecompressor.obj
 0003:00000170       ?_OptionsStorage@?1??__local_stdio_printf_options@@9@4_KA 10006170     imageDecompressor.obj
 0003:00000178       ?memory_map_image@ImageFileReader@@0_NA 10006178     imageFile.obj
 0003:0000017c       ?_reader_table_lock@@3VSimpleCriticalSection@@A 1000617c     imageFile.obj
 0003:00000194       ?_reader_table@ImageFileReader@@0VImageFileReaderTable@@A 10006194     imageFile.obj
 0003:000004c0       ?__type_info_root_node@@3U__type_info_node@@A 100064c0     MSVCRT:tncleanup.obj
 0003:000004c8       ?_OptionsStorage@?1??__local_stdio_scanf_options@@9@4_KA 100064c8     MSVCRT:default_local_stdio_options.obj
 0003:000004d0       ___scrt_current_native_startup_state 100064d0     MSVCRT:utility.obj
 0003:000004d4       ___scrt_native_startup_lock 100064d4     MSVCRT:utility.obj
 0003:000004f4       ___scrt_debugger_hook_flag 100064f4     MSVCRT:utility_desktop.obj
 0003:000004f8       ___isa_available           100064f8     MSVCRT:cpu_disp.obj
 0003:000004fc       ___favor                   100064fc     MSVCRT:cpu_disp.obj
 0003:00000500       ___dyn_tls_init_callback   10006500     <common>

 entry point at        0001:00001acb

 Static symbols

 0000:ffff7000       .debug$S                   10000000     jimage.exp
 0000:ffff7000       .debug$S                   10000000     vcruntime:VCRUNTIME140.dll
 0000:ffff7000       .debug$S                   10000000     vcruntime:VCRUNTIME140.dll
 0000:ffff7000       .debug$S                   10000000     vcruntime:VCRUNTIME140.dll
 0000:ffff7000       .debug$S                   10000000     vcruntime:VCRUNTIME140.dll
 0000:ffff7000       .debug$S                   10000000     vcruntime:VCRUNTIME140.dll
 0000:ffff7000       .debug$S                   10000000     vcruntime:VCRUNTIME140.dll
 0000:ffff7000       .debug$S                   10000000     vcruntime:VCRUNTIME140.dll
 0000:ffff7000       .debug$S                   10000000     vcruntime:VCRUNTIME140.dll
 0000:ffff7000       .debug$S                   10000000     vcruntime:VCRUNTIME140.dll
 0000:ffff7000       .debug$S                   10000000     vcruntime:VCRUNTIME140.dll
 0000:ffff7000       .debug$S                   10000000     ucrt:api-ms-win-crt-filesystem-l1-1-0.dll
 0000:ffff7000       .debug$S                   10000000     ucrt:api-ms-win-crt-heap-l1-1-0.dll
 0000:ffff7000       .debug$S                   10000000     ucrt:api-ms-win-crt-heap-l1-1-0.dll
 0000:ffff7000       .debug$S                   10000000     ucrt:api-ms-win-crt-heap-l1-1-0.dll
 0000:ffff7000       .debug$S                   10000000     ucrt:api-ms-win-crt-heap-l1-1-0.dll
 0000:ffff7000       .debug$S                   10000000     ucrt:api-ms-win-crt-heap-l1-1-0.dll
 0000:ffff7000       .debug$S                   10000000     ucrt:api-ms-win-crt-runtime-l1-1-0.dll
 0000:ffff7000       .debug$S                   10000000     ucrt:api-ms-win-crt-runtime-l1-1-0.dll
 0000:ffff7000       .debug$S                   10000000     ucrt:api-ms-win-crt-runtime-l1-1-0.dll
 0000:ffff7000       .debug$S                   10000000     ucrt:api-ms-win-crt-runtime-l1-1-0.dll
 0000:ffff7000       .debug$S                   10000000     ucrt:api-ms-win-crt-runtime-l1-1-0.dll
 0000:ffff7000       .debug$S                   10000000     ucrt:api-ms-win-crt-runtime-l1-1-0.dll
 0000:ffff7000       .debug$S                   10000000     ucrt:api-ms-win-crt-runtime-l1-1-0.dll
 0000:ffff7000       .debug$S                   10000000     ucrt:api-ms-win-crt-runtime-l1-1-0.dll
 0000:ffff7000       .debug$S                   10000000     ucrt:api-ms-win-crt-runtime-l1-1-0.dll
 0000:ffff7000       .debug$S                   10000000     ucrt:api-ms-win-crt-runtime-l1-1-0.dll
 0000:ffff7000       .debug$S                   10000000     ucrt:api-ms-win-crt-runtime-l1-1-0.dll
 0000:ffff7000       .debug$S                   10000000     ucrt:api-ms-win-crt-runtime-l1-1-0.dll
 0000:ffff7000       .debug$S                   10000000     ucrt:api-ms-win-crt-stdio-l1-1-0.dll
 0000:ffff7000       .debug$S                   10000000     ucrt:api-ms-win-crt-stdio-l1-1-0.dll
 0000:ffff7000       .debug$S                   10000000     ucrt:api-ms-win-crt-stdio-l1-1-0.dll
 0000:ffff7000       .debug$S                   10000000     ucrt:api-ms-win-crt-stdio-l1-1-0.dll
 0000:ffff7000       .debug$S                   10000000     ucrt:api-ms-win-crt-stdio-l1-1-0.dll
 0000:ffff7000       .debug$S                   10000000     ucrt:api-ms-win-crt-string-l1-1-0.dll
 0000:ffff7000       .debug$S                   10000000     ucrt:api-ms-win-crt-string-l1-1-0.dll
 0000:ffff7000       .debug$S                   10000000     ucrt:api-ms-win-crt-string-l1-1-0.dll
 0000:ffff7000       .debug$S                   10000000     ucrt:api-ms-win-crt-string-l1-1-0.dll
 0000:ffff7000       .debug$S                   10000000     ucrt:api-ms-win-crt-string-l1-1-0.dll
 0000:ffff7000       .debug$S                   10000000     kernel32:KERNEL32.dll
 0000:ffff7000       .debug$S                   10000000     kernel32:KERNEL32.dll
 0000:ffff7000       .debug$S                   10000000     kernel32:KERNEL32.dll
 0000:ffff7000       .debug$S                   10000000     kernel32:KERNEL32.dll
 0000:ffff7000       .debug$S                   10000000     kernel32:KERNEL32.dll
 0000:ffff7000       .debug$S                   10000000     kernel32:KERNEL32.dll
 0000:ffff7000       .debug$S                   10000000     kernel32:KERNEL32.dll
 0000:ffff7000       .debug$S                   10000000     kernel32:KERNEL32.dll
 0000:ffff7000       .debug$S                   10000000     kernel32:KERNEL32.dll
 0000:ffff7000       .debug$S                   10000000     kernel32:KERNEL32.dll
 0000:ffff7000       .debug$S                   10000000     kernel32:KERNEL32.dll
 0000:ffff7000       .debug$S                   10000000     kernel32:KERNEL32.dll
 0000:ffff7000       .debug$S                   10000000     kernel32:KERNEL32.dll
 0000:ffff7000       .debug$S                   10000000     kernel32:KERNEL32.dll
 0000:ffff7000       .debug$S                   10000000     kernel32:KERNEL32.dll
 0000:ffff7000       .debug$S                   10000000     kernel32:KERNEL32.dll
 0000:ffff7000       .debug$S                   10000000     kernel32:KERNEL32.dll
 0000:ffff7000       .debug$S                   10000000     kernel32:KERNEL32.dll
 0000:ffff7000       .debug$S                   10000000     kernel32:KERNEL32.dll
 0000:ffff7000       .debug$S                   10000000     kernel32:KERNEL32.dll
 0000:ffff7000       .debug$S                   10000000     kernel32:KERNEL32.dll
 0000:ffff7000       .debug$S                   10000000     kernel32:KERNEL32.dll
 0000:ffff7000       .debug$S                   10000000     kernel32:KERNEL32.dll
 0000:ffff7000       .debug$S                   10000000     kernel32:KERNEL32.dll
 0000:ffff7000       .debug$S                   10000000     kernel32:KERNEL32.dll
 0000:ffff7000       .debug$S                   10000000     kernel32:KERNEL32.dll
 0001:00000000       ??__E?_reader_table@ImageFileReader@@0VImageFileReaderTable@@A@@YAXXZ 10001000 f   imageFile.obj
 0001:0000000a       ??__E_reader_table_lock@@YAXXZ 1000100a f   imageFile.obj
 0001:00001760       $$000000                   10002760     MSVCRT:chkstk.obj
 0001:00001774       cs10                       10002774     MSVCRT:chkstk.obj
 0001:00001782       cs20                       10002782     MSVCRT:chkstk.obj
 0001:0000178b       ?dllmain_crt_dispatch@@YGHQAUHINSTANCE__@@KQAX@Z 1000278b f   MSVCRT:dll_dllmain.obj
 0001:000017de       ?dllmain_crt_process_attach@@YAHQAUHINSTANCE__@@QAX@Z 100027de f   MSVCRT:dll_dllmain.obj
 0001:000018e5       ?dllmain_crt_process_detach@@YAH_N@Z 100028e5 f   MSVCRT:dll_dllmain.obj
 0001:00001995       ?dllmain_dispatch@@YAHQAUHINSTANCE__@@KQAX@Z 10002995 f   MSVCRT:dll_dllmain.obj
 0001:00001aa0       ?dllmain_raw@@YGHQAUHINSTANCE__@@KQAX@Z 10002aa0 f   MSVCRT:dll_dllmain.obj
 0001:00001c0a       ___get_entropy             10002c0a f   MSVCRT:gs_support.obj
 0001:00001cff       ?find_pe_section@@YAPAU_IMAGE_SECTION_HEADER@@QAEI@Z 10002cff f   MSVCRT:utility.obj
 0001:00002160       $$000000                   10003160     MSVCRT:sehprolg4.obj
 0002:00000104       ??_reader_table$initializer$@ImageFileReader@@0P6AXXZA@@3P6AXXZA 10004104     imageFile.obj
 0002:00000108       ?_reader_table_lock$initializer$@@3P6AXXZA 10004108     imageFile.obj
 0002:00000238       _GS_ExceptionPointers      10004238     MSVCRT:gs_report.obj
 0002:00000a38       __sehtable$?dllmain_crt_process_attach@@YAHQAUHINSTANCE__@@QAX@Z 10004a38     MSVCRT:dll_dllmain.obj
 0002:00000a58       __sehtable$?dllmain_crt_process_detach@@YAH_N@Z 10004a58     MSVCRT:dll_dllmain.obj
 0002:00000a80       __sehtable$?dllmain_dispatch@@YAHQAUHINSTANCE__@@KQAX@Z 10004a80     MSVCRT:dll_dllmain.obj
 0002:00000b30       __sehtable$___scrt_is_nonwritable_in_current_image 10004b30     MSVCRT:utility.obj
 0002:00000b50       .edata                     10004b50     jimage.exp
 0002:00000b78       rgpv                       10004b78     jimage.exp
 0002:00000b94       rgszName                   10004b94     jimage.exp
 0002:00000bb0       rgwOrd                     10004bb0     jimage.exp
 0002:00000bbe       szName                     10004bbe     jimage.exp
 0002:00000bc9       $N00001                    10004bc9     jimage.exp
 0002:00000bd6       $N00002                    10004bd6     jimage.exp
 0002:00000bea       $N00003                    10004bea     jimage.exp
 0002:00000bfd       $N00004                    10004bfd     jimage.exp
 0002:00000c09       $N00005                    10004c09     jimage.exp
 0002:00000c20       $N00006                    10004c20     jimage.exp
 0002:00000c38       $N00007                    10004c38     jimage.exp
 0002:00001014       .idata$6                   10005014     kernel32:KERNEL32.dll
 0002:000010b8       .idata$6                   100050b8     vcruntime:VCRUNTIME140.dll
 0002:00001232       .idata$6                   10005232     ucrt:api-ms-win-crt-stdio-l1-1-0.dll
 0002:00001252       .idata$6                   10005252     ucrt:api-ms-win-crt-string-l1-1-0.dll
 0002:00001274       .idata$6                   10005274     ucrt:api-ms-win-crt-heap-l1-1-0.dll
 0002:00001294       .idata$6                   10005294     ucrt:api-ms-win-crt-filesystem-l1-1-0.dll
 0002:000012ba       .idata$6                   100052ba     ucrt:api-ms-win-crt-runtime-l1-1-0.dll
 0003:00000168       ?ZipInflateFully@@3P6AEPAX_J01PAPAD@ZA 10006168     imageDecompressor.obj
 0003:000001a0       _GS_ExceptionRecord        100061a0     MSVCRT:gs_report.obj
 0003:000001f0       _GS_ContextRecord          100061f0     MSVCRT:gs_report.obj
 0003:000004bc       ?__proc_attached@@3HA      100064bc     MSVCRT:dll_dllmain.obj
 0003:000004d8       ?is_initialized_as_dll@@3_NA 100064d8     MSVCRT:utility.obj
 0003:000004d9       ?module_local_atexit_table_initialized@@3_NA 100064d9     MSVCRT:utility.obj
 0003:000004dc       ?module_local_atexit_table@@3U_onexit_table_t@@A 100064dc     MSVCRT:utility.obj
 0003:000004e8       ?module_local_at_quick_exit_table@@3U_onexit_table_t@@A 100064e8     MSVCRT:utility.obj
 0004:00000060       $R000000                   10007060     jimage.dll.res
